******************************************************************************
TMS470R1x COFF vLinker                           Version 1.9902
******************************************************************************
>> Linked Thu Mar 30 20:06:43 2006

OUTPUT FILE NAME:   <W:\_Out\bin\LangPack\HYPB1AL1200025.out>
ENTRY POINT SYMBOL: "_LanguagePack"  address: 01170000


MEMORY CONFIGURATION

                  name            origin    length      used    attr    fill
         ----------------------  --------  ---------  --------  ----  --------
         LP_MEM                  01170000  0001c0000  0011817c  R IX
         LP_MEM2                 01330000  000250000  00241a24  R IX


SECTION ALLOCATION MAP

 output                                  attributes/
section   page    origin      length       input sections
--------  ----  ----------  ----------   ----------------
___page_info__
        0    00000000    00000008     DSECT
                  00000000    00000008     --PAGE INFORMATION--

___section_info__
        0    00000000    00000008     DSECT
                  00000000    00000008     --SECTION INFORMATION--

.langpack
        0    01170000    00000028     
                  01170000    00000028     mmi_lang_pack.obj (.langpack)

.const  0    01170028    00118154     
                  01170028    00017550     LangPack.lib : lp_Finnish_Dict (.const)
                  01187578    0001305c     openwave_wap3.lib : rescomn.o (.const)
                  0119a5d4    0000dd58     LangPack.lib : lp_Swedish_Dict (.const)
                  011a832c    0000dcf0                  : lp_Norwegian_Di (.const)
                  011b601c    0000dcdc                  : lp_Danish_Dict. (.const)
                  011c3cf8    0000dcac                  : lp_Dutch_Dict.o (.const)
                  011d19a4    0000c390                  : lp_German_Dict. (.const)
                  011ddd34    0000c124                  : lp_Latin_Font.o (.const)
                  011e9e58    0000b884                  : lp_Finnish_Text (.const)
                  011f56dc    0000b558                  : lp_German_Text. (.const)
                  01200c34    0000b500                  : lp_French_Dict. (.const)
                  0120c134    0000b16c                  : lp_French_Text. (.const)
                  012172a0    0000b030                  : lp_Dutch_Text.o (.const)
                  012222d0    0000a9c0                  : lp_Swedish_Text (.const)
                  0122cc90    0000a97c                  : lp_Norwegian_Te (.const)
                  0123760c    0000a89c                  : lp_Danish_Text. (.const)
                  01241ea8    0000a224                  : lp_English_Text (.const)
                  0124c0cc    00009078                  : lp_English_Dict (.const)
                  01255144    00006710     openwave_wap3.lib : resdede.o (.const)
                  0125b854    00006324                       : resfrfr.o (.const)
                  01261b78    00005fdc                       : resnlnl.o (.const)
                  01267b54    00005db8                       : resfifi.o (.const)
                  0126d90c    00005c70                       : ressvse.o (.const)
                  0127357c    000059e4                       : resdadk.o (.const)
                  01278f60    000058ac                       : resnono.o (.const)
                  0127e80c    0000543c                       : resen.o (.const)
                  01283c48    00001f48     LangPack.lib : img_name.obj (.const)
                  01285b90    000015b4                  : melody_name.obj (.const)
                  01287144    00000370                  : mmi_ime_info.ob (.const)
                  012874b4    0000023c     mmi_lang_data.obj (.const)
                  012876f0    00000150     LangPack.lib : wap_French_User (.const)
                  01287840    00000140                  : wap_German_User (.const)
                  01287980    00000134                  : wap_Dutch_UserL (.const)
                  01287ab4    0000012c                  : wap_English_Use (.const)
                  01287be0    00000128                  : wap_Finnish_Use (.const)
                  01287d08    00000124                  : wap_Swedish_Use (.const)
                  01287e2c    00000120                  : wap_Danish_User (.const)
                  01287f4c    0000011c                  : wap_Norwegian_U (.const)
                  01288068    00000094                  : lp_CP1252_Encod (.const)
                  012880fc    0000005c                  : lp_CP1252_Decod (.const)
                  01288158    00000024     mmi_lang_pack.obj (.const)

.text   0    0128817c    00000000     UNINITIALIZED

.media  0    01330000    00241a24     
                  01330000    002129c4     Media.lib : img_data.obj (.const)
                  015429c4    0002f060               : melody_data.obj (.const)


GLOBAL SYMBOLS: SORTED ALPHABETICALLY BY Name 

address    name
--------   ----
0128817c   .text
01287144   _IME_MODULES
01287660   _LANG_INFO_DANISH
012875e0   _LANG_INFO_DUTCH
01287520   _LANG_INFO_ENGLISH
012876a0   _LANG_INFO_FINNISH
012875a0   _LANG_INFO_FRENCH
01287560   _LANG_INFO_GERMAN
012876e0   _LANG_INFO_NORWEGIAN
01287620   _LANG_INFO_SWEDISH
01170000   _LanguagePack
0128817c   ___etext__
0128817c   ___text__
0118980c   _aboutTIL
01189a68   _aboutsslTIL
0118967c   _advancedTIL
0118b50c   _advdmenuTIL
01189ed0   _alertTIL
0118a0d0   _alert_0TIL
0118a30c   _alert_imTIL
01195114   _alertdlgTIL
0118b6f0   _altadvdTIL
01188358   _altsettTIL
01187b8c   _apperrTIL
0118a4ec   _aspawnTIL
0118a584   _authTIL
0118af58   _bawalletTIL
0118c73c   _bkmkmenuTIL
01191d24   _bktbmptyTIL
01187578   _blankTIL
01190c1c   _bookccf2TIL
0118e398   _bookccfmTIL
0118d590   _bookdelTIL
0118e784   _bookdelaTIL
0118fd74   _bookdtlTIL
0118d708   _bookerrTIL
011909c4   _bookfdlsTIL
01190888   _bookffulTIL
01190318   _bookfldlTIL
0118f308   _bookflhkTIL
0118dd24   _bookfolTIL
01190604   _bookfullTIL
0118d82c   _bookgoTIL
0118f620   _bookhtkyTIL
01191fd8   _bookinpoTIL
0118e978   _bookmkpgTIL
01190764   _bookmmsgTIL
0118e4b8   _bookmoveTIL
0118fbcc   _bookmtnfTIL
01190f18   _bookmvflTIL
01191320   _bookmvtpTIL
0118c7e0   _booknewTIL
0118da5c   _booknewfTIL
01190d98   _booknomkTIL
0119185c   _bookpassTIL
01191e8c   _bookpostTIL
01191988   _bookpserTIL
0118cadc   _booksavdTIL
01191ad4   _booksaveTIL
0118ec28   _bookstfTIL
0118fa18   _bookstnfTIL
0118ccb8   _booktopTIL
0118ff18   _booktpdlTIL
0118ef20   _booktphkTIL
0118cc28   _bookwrapTIL
UNDEFED _c_int00
01197fbc   _camgmtTIL
01194e28   _cctlingrTIL
01194c24   _cctprmptTIL
01197e74   _certerb0TIL
01197b78   _certerbTIL
01197774   _certinfoTIL
011979f4   _certnoneTIL
0118bb6c   _clearTIL
0118be2c   _clearpopTIL
0119522c   _confdlgTIL
0119867c   _connprmtTIL
0119887c   _connsec0TIL
0119895c   _connsec1TIL
01198a30   _connsec2TIL
01188b0c   _cookiclrTIL
01188ec0   _cryptTIL
01199f84   _devpopu1TIL
01199f14   _devpopupTIL
01199fcc   _devpulldTIL
0118c280   _dialogTIL
01196180   _dldoneTIL
011963b8   _dlerror2TIL
01196218   _dlerrorTIL
01196350   _dlprogresTIL
01196284   _dlpromptTIL
0118c4dc   _drmmsgTIL
011960e0   _e2eexpTIL
011960a8   _e2einvalTIL
01187ebc   _entrhomeTIL
011955d0   _gotourlTIL
0118ab38   _histlistTIL
0118a778   _histnavTIL
0118bfb0   _histpopTIL
0118b110   _homeexitTIL
01187e0c   _homepickTIL
0118b20c   _homesvdTIL
01196070   _httperrTIL
0119279c   _httprefTIL
01570fc4   _i_Accessary_In
01569788   _i_Alert_1
0156a900   _i_Alert_10
0156ab08   _i_Alert_11
0156ac5c   _i_Alert_12
0156984c   _i_Alert_2
01569958   _i_Alert_3
01569b38   _i_Alert_4
01569f64   _i_Alert_5
0156a070   _i_Alert_6
0156a314   _i_Alert_7
0156a3d8   _i_Alert_8
0156a7e8   _i_Alert_9
01571094   _i_Battery_Low
01545728   _i_BenQisComing
01562ca8   _i_Breeze
01570a74   _i_CMR_MutiShot
01570924   _i_CMR_Timer_Long
0157084c   _i_CMR_Timer_Short
015711a8   _i_Call_Start
0156b3bc   _i_Camera_Record_End
0156c574   _i_Camera_Record_Start
0156478c   _i_Dance
01546694   _i_DownHome
01339090   _i_EMS_Angry
01571874   _i_EMS_Bugle
01571308   _i_EMS_Chimes_High
015713a0   _i_EMS_Chimes_Low
01571770   _i_EMS_ChordHigh
015717f4   _i_EMS_ChordLow
0157165c   _i_EMS_Claps
01337878   _i_EMS_Confused
01333c3c   _i_EMS_Crying
0133a8a8   _i_EMS_Devil
0157143c   _i_EMS_Ding
015715c4   _i_EMS_Drum
015716e8   _i_EMS_Fanfare
01330000   _i_EMS_Flirty
01330c0c   _i_EMS_Glad
01339c9c   _i_EMS_Glasses
01336060   _i_EMS_Indifferent
01336c6c   _i_EMS_Kissing
01335454   _i_EMS_Laughing
0133b7c0   _i_EMS_NoDefAnim
0133b4b4   _i_EMS_NoDefPic
0133bacc   _i_EMS_NoDefSound
01571538   _i_EMS_Notify
0133bea4   _i_EMS_Paw
01332424   _i_EMS_Sad
01331818   _i_EMS_Sceptic
0133bb98   _i_EMS_Star
015714bc   _i_EMS_Tada
01338484   _i_EMS_Tongue
0133c1b0   _i_EMS_TurnAround
01334848   _i_EMS_Winking
01333030   _i_EMS_Wow
0155433c   _i_Fire
0154ce48   _i_Fly
01559e7c   _i_Friendship
01555934   _i_LadyMary
01571220   _i_Network_On
015680dc   _i_Papillon
01570754   _i_Power_Down
015704d8   _i_Power_Up
0156d72c   _i_SelfTimer_1Seconds1beat
0156e58c   _i_SelfTimer_1Seconds3beat
0154fbc0   _i_Shopping
015718f8   _i_ShotTone1
01571900   _i_ShotTone2
01571908   _i_ShotTone3
01571910   _i_ShotTone4
01571918   _i_ShotTone5
0156ad74   _i_ShotTone_Multishot
01548814   _i_Soul
01557824   _i_Speed
0155fb9c   _i_SunnySamba
01570f38   _i_Vedio_Record_End
01570ebc   _i_Vedio_Record_Start
015429c4   _i_aroundtheworld
0154b6e0   _i_straightway
01195dc8   _imageTIL
01195e24   _imgdispTIL
01195ac4   _imginfoTIL
01195978   _imgmenuTIL
0118c230   _intrlcssTIL
0118918c   _keycheckTIL
01189200   _keytimeTIL
011950b4   _loopTIL
012880fc   _lp_CP1252_Decode
01288068   _lp_CP1252_Encode
011b601c   _lp_Danish_Dict
01287630   _lp_Danish_ResList
01241e9c   _lp_Danish_Text
011c3cf8   _lp_Dutch_Dict
012875b0   _lp_Dutch_ResList
012222c4   _lp_Dutch_Text
0124c0cc   _lp_English_Dict
012874f0   _lp_English_ResList
0124c0c0   _lp_English_Text
01170028   _lp_Finnish_Dict
01287670   _lp_Finnish_ResList
011f56d0   _lp_Finnish_Text
01200c34   _lp_French_Dict
01287570   _lp_French_ResList
01217294   _lp_French_Text
011d19a4   _lp_German_Dict
01287530   _lp_German_ResList
01200c28   _lp_German_Text
012874e4   _lp_Global_LangResList
012874b4   _lp_Global_ResList
011ddd34   _lp_Latin_Font
011a832c   _lp_Norwegian_Dict
012876b0   _lp_Norwegian_ResList
01237600   _lp_Norwegian_Text
0119a5d4   _lp_Swedish_Dict
012875f0   _lp_Swedish_ResList
0122cc84   _lp_Swedish_Text
01192124   _markcss2TIL
015417f4   _ml_imageLib
012849c0   _ml_imageNameLib
01571920   _ml_melodyLib
01287040   _ml_melodyNameLib
011953dc   _mmccomptTIL
011952f0   _mmcconfmTIL
01195390   _mmcdispTIL
01195428   _mmcerrorTIL
011975e0   _mmsImmRetrievalTIL
011976a8   _mmssplashTIL
01286c00   _n_Alert_1
01286d20   _n_Alert_10
01285e44   _n_Alert_10_e
01286758   _n_Alert_10_fren
012862dc   _n_Alert_10_germ
01286d40   _n_Alert_11
01285e58   _n_Alert_11_e
0128676c   _n_Alert_11_fren
012862f0   _n_Alert_11_germ
01286d60   _n_Alert_12
01285e6c   _n_Alert_12_e
01286780   _n_Alert_12_fren
01286304   _n_Alert_12_germ
01285db4   _n_Alert_1_e
012866a4   _n_Alert_1_fren
0128624c   _n_Alert_1_germ
01286c20   _n_Alert_2
01285dc4   _n_Alert_2_e
012866b8   _n_Alert_2_fren
0128625c   _n_Alert_2_germ
01286c40   _n_Alert_3
01285dd4   _n_Alert_3_e
012866cc   _n_Alert_3_fren
0128626c   _n_Alert_3_germ
01286c60   _n_Alert_4
01285de4   _n_Alert_4_e
012866e0   _n_Alert_4_fren
0128627c   _n_Alert_4_germ
01286c80   _n_Alert_5
01285df4   _n_Alert_5_e
012866f4   _n_Alert_5_fren
0128628c   _n_Alert_5_germ
01286ca0   _n_Alert_6
01285e04   _n_Alert_6_e
01286708   _n_Alert_6_fren
0128629c   _n_Alert_6_germ
01286cc0   _n_Alert_7
01285e14   _n_Alert_7_e
0128671c   _n_Alert_7_fren
012862ac   _n_Alert_7_germ
01286ce0   _n_Alert_8
01285e24   _n_Alert_8_e
01286730   _n_Alert_8_fren
012862bc   _n_Alert_8_germ
01286d00   _n_Alert_9
01285e34   _n_Alert_9_e
01286744   _n_Alert_9_fren
012862cc   _n_Alert_9_germ
01286ba0   _n_BeautifulGirls
01285d54   _n_BeautifulGirls_e
01286644   _n_BeautifulGirls_fren
012861ec   _n_BeautifulGirls_germ
01286920   _n_BenQisComing
01285bb4   _n_BenQisComing_e
01286488   _n_BenQisComing_fren
01286058   _n_BenQisComing_germ
01286a80   _n_Breeze
01285c7c   _n_Breeze_e
0128656c   _n_Breeze_fren
01286114   _n_Breeze_germ
012847c0   _n_COM_Wallpaper1
01283e50   _n_COM_Wallpaper1_e
01284428   _n_COM_Wallpaper1_fren
01284174   _n_COM_Wallpaper1_germ
012847e0   _n_COM_Wallpaper2
01283e64   _n_COM_Wallpaper2_e
0128443c   _n_COM_Wallpaper2_fren
01284188   _n_COM_Wallpaper2_germ
01284800   _n_COM_Wallpaper3
01283e7c   _n_COM_Wallpaper3_e
01284454   _n_COM_Wallpaper3_fren
012841a0   _n_COM_Wallpaper3_germ
01284820   _n_COM_Wallpaper4
01283e90   _n_COM_Wallpaper4_e
01284468   _n_COM_Wallpaper4_fren
012841b4   _n_COM_Wallpaper4_germ
01284840   _n_COM_Wallpaper5
01283ea4   _n_COM_Wallpaper5_e
0128447c   _n_COM_Wallpaper5_fren
012841c8   _n_COM_Wallpaper5_germ
01286aa0   _n_Dance
01285c8c   _n_Dance_e
0128657c   _n_Dance_fren
01286124   _n_Dance_germ
01286940   _n_DownHome
01285bc8   _n_DownHome_e
0128649c   _n_DownHome_fren
01286068   _n_DownHome_germ
012846a0   _n_EMS_Angry
01283d98   _n_EMS_Angry_e
01284374   _n_EMS_Angry_fren
012840b4   _n_EMS_Angry_germ
01286f80   _n_EMS_Bugle
01285fb0   _n_EMS_Bugle_e
01286878   _n_EMS_Bugle_fren
012863e4   _n_EMS_Bugle_germ
01286d80   _n_EMS_Chimes_High
01285e80   _n_EMS_Chimes_High_e
01286794   _n_EMS_Chimes_High_fren
01286318   _n_EMS_Chimes_High_germ
01286da0   _n_EMS_Chimes_Low
01285e98   _n_EMS_Chimes_Low_e
012867b4   _n_EMS_Chimes_Low_fren
01286330   _n_EMS_Chimes_Low_germ
01286e80   _n_EMS_ChordHigh
01285f00   _n_EMS_ChordHigh_e
01286834   _n_EMS_ChordHigh_fren
012863a4   _n_EMS_ChordHigh_germ
01286ea0   _n_EMS_ChordLow
01285f14   _n_EMS_ChordLow_e
0128684c   _n_EMS_ChordLow_fren
012863b8   _n_EMS_ChordLow_germ
01286e40   _n_EMS_Claps
01285ee4   _n_EMS_Claps_e
01286810   _n_EMS_Claps_fren
01286380   _n_EMS_Claps_germ
01284660   _n_EMS_Confused
01283d54   _n_EMS_Confused_e
01284344   _n_EMS_Confused_fren
01284068   _n_EMS_Confused_germ
012845c0   _n_EMS_Crying
01283cc0   _n_EMS_Crying_e
012842c4   _n_EMS_Crying_fren
01283fe8   _n_EMS_Crying_germ
012846e0   _n_EMS_Devil
01283dd0   _n_EMS_Devil_e
01284394   _n_EMS_Devil_fren
012840f0   _n_EMS_Devil_germ
01286dc0   _n_EMS_Ding
01285eb0   _n_EMS_Ding_e
012867d0   _n_EMS_Ding_fren
01286348   _n_EMS_Ding_germ
01286e20   _n_EMS_Drum
01285ed8   _n_EMS_Drum_e
012867fc   _n_EMS_Drum_fren
01286370   _n_EMS_Drum_germ
01286e60   _n_EMS_Fanfare
01285ef0   _n_EMS_Fanfare_e
01286824   _n_EMS_Fanfare_fren
01286394   _n_EMS_Fanfare_germ
01284520   _n_EMS_Flirty
01283c48   _n_EMS_Flirty_e
0128426c   _n_EMS_Flirty_fren
01283f48   _n_EMS_Flirty_germ
01284540   _n_EMS_Glad
01283c70   _n_EMS_Glad_e
01284280   _n_EMS_Glad_fren
01283f78   _n_EMS_Glad_germ
012846c0   _n_EMS_Glasses
01283db0   _n_EMS_Glasses_e
01284380   _n_EMS_Glasses_fren
012840d4   _n_EMS_Glasses_germ
01284620   _n_EMS_Indifferent
01283d10   _n_EMS_Indifferent_e
01284304   _n_EMS_Indifferent_fren
0128402c   _n_EMS_Indifferent_germ
01284640   _n_EMS_Kissing
01283d34   _n_EMS_Kissing_e
0128431c   _n_EMS_Kissing_fren
01284048   _n_EMS_Kissing_germ
01284600   _n_EMS_Laughing
01283cf4   _n_EMS_Laughing_e
012842f8   _n_EMS_Laughing_fren
01284018   _n_EMS_Laughing_germ
01284720   _n_EMS_NoDefAnim
01283df4   _n_EMS_NoDefAnim_e
012843bc   _n_EMS_NoDefAnim_fren
01284118   _n_EMS_NoDefAnim_germ
01284700   _n_EMS_NoDefPic
01283ddc   _n_EMS_NoDefPic_e
012843a4   _n_EMS_NoDefPic_fren
01284100   _n_EMS_NoDefPic_germ
01284740   _n_EMS_NoDefSound
01283e10   _n_EMS_NoDefSound_e
012843d8   _n_EMS_NoDefSound_fren
01284134   _n_EMS_NoDefSound_germ
01286e00   _n_EMS_Notify
01285ec8   _n_EMS_Notify_e
012867e8   _n_EMS_Notify_fren
01286360   _n_EMS_Notify_germ
01284780   _n_EMS_Paw
01283e30   _n_EMS_Paw_e
012843fc   _n_EMS_Paw_fren
01284154   _n_EMS_Paw_germ
01284580   _n_EMS_Sad
01283ca0   _n_EMS_Sad_e
012842a4   _n_EMS_Sad_fren
01283fbc   _n_EMS_Sad_germ
01284560   _n_EMS_Sceptic
01283c84   _n_EMS_Sceptic_e
01284290   _n_EMS_Sceptic_fren
01283f98   _n_EMS_Sceptic_germ
01284760   _n_EMS_Star
01283e24   _n_EMS_Star_e
012843ec   _n_EMS_Star_fren
01284148   _n_EMS_Star_germ
01286de0   _n_EMS_Tada
01285ebc   _n_EMS_Tada_e
012867dc   _n_EMS_Tada_fren
01286354   _n_EMS_Tada_germ
01284680   _n_EMS_Tongue
01283d70   _n_EMS_Tongue_e
01284358   _n_EMS_Tongue_fren
0128408c   _n_EMS_Tongue_germ
012847a0   _n_EMS_TurnAround
01283e38   _n_EMS_TurnAround_e
01284408   _n_EMS_TurnAround_fren
01284160   _n_EMS_TurnAround_germ
012845e0   _n_EMS_Winking
01283cd8   _n_EMS_Winking_e
012842d4   _n_EMS_Winking_fren
01283ffc   _n_EMS_Winking_germ
012845a0   _n_EMS_Wow
01283cb4   _n_EMS_Wow_e
012842b4   _n_EMS_Wow_fren
01283fdc   _n_EMS_Wow_germ
012869e0   _n_Fire
01285c20   _n_Fire_e
01286510   _n_Fire_fren
012860b8   _n_Fire_germ
012869a0   _n_Fly
01285c04   _n_Fly_e
012864f4   _n_Fly_fren
0128609c   _n_Fly_germ
01286a40   _n_Friendship
01285c4c   _n_Friendship_e
0128653c   _n_Friendship_fren
012860e4   _n_Friendship_germ
01286ae0   _n_GlistensTheQuartz
01285cac   _n_GlistensTheQuartz_e
0128659c   _n_GlistensTheQuartz_fren
01286144   _n_GlistensTheQuartz_germ
01286b00   _n_GrandfathersClock
01285cd4   _n_GrandfathersClock_e
012865c4   _n_GrandfathersClock_fren
0128616c   _n_GrandfathersClock_germ
01286bc0   _n_GreatPalace
01285d74   _n_GreatPalace_e
01286664   _n_GreatPalace_fren
0128620c   _n_GreatPalace_germ
01286a00   _n_LadyMary
01285c2c   _n_LadyMary_e
0128651c   _n_LadyMary_fren
012860c4   _n_LadyMary_germ
01286b60   _n_Nostalgia
01285d28   _n_Nostalgia_e
01286618   _n_Nostalgia_fren
012861c0   _n_Nostalgia_germ
01286ac0   _n_Papillon
01285c98   _n_Papillon_e
01286588   _n_Papillon_fren
01286130   _n_Papillon_germ
01286b20   _n_RedIsTheRose
01285cfc   _n_RedIsTheRose_e
012865ec   _n_RedIsTheRose_fren
01286194   _n_RedIsTheRose_germ
01284860   _n_SHRCT_Boy
01283eb0   _n_SHRCT_Boy_e
01284488   _n_SHRCT_Boy_fren
012841d4   _n_SHRCT_Boy_germ
01284880   _n_SHRCT_Brother
01283eb8   _n_SHRCT_Brother_e
01284490   _n_SHRCT_Brother_fren
012841dc   _n_SHRCT_Brother_germ
012848a0   _n_SHRCT_Father
01283ec8   _n_SHRCT_Father_e
012844a0   _n_SHRCT_Father_fren
012841ec   _n_SHRCT_Father_germ
012848c0   _n_SHRCT_Girl
01283ed8   _n_SHRCT_Girl_e
012844b0   _n_SHRCT_Girl_fren
012841fc   _n_SHRCT_Girl_germ
012848e0   _n_SHRCT_Grandma
01283ee4   _n_SHRCT_Grandma_e
012844bc   _n_SHRCT_Grandma_fren
01284208   _n_SHRCT_Grandma_germ
01284900   _n_SHRCT_Grandpa
01283ef4   _n_SHRCT_Grandpa_e
012844cc   _n_SHRCT_Grandpa_fren
01284218   _n_SHRCT_Grandpa_germ
01284920   _n_SHRCT_Man
01283f04   _n_SHRCT_Man_e
012844dc   _n_SHRCT_Man_fren
01284228   _n_SHRCT_Man_germ
01284940   _n_SHRCT_Mother
01283f0c   _n_SHRCT_Mother_e
012844e4   _n_SHRCT_Mother_fren
01284230   _n_SHRCT_Mother_germ
01284960   _n_SHRCT_Nobody
01283f1c   _n_SHRCT_Nobody_e
012844f4   _n_SHRCT_Nobody_fren
01284240   _n_SHRCT_Nobody_germ
01284980   _n_SHRCT_Sister
01283f2c   _n_SHRCT_Sister_e
01284504   _n_SHRCT_Sister_fren
01284250   _n_SHRCT_Sister_germ
012849a0   _n_SHRCT_Woman
01283f3c   _n_SHRCT_Woman_e
01284514   _n_SHRCT_Woman_fren
01284260   _n_SHRCT_Woman_germ
012869c0   _n_Shopping
01285c0c   _n_Shopping_e
012864fc   _n_Shopping_fren
012860a4   _n_Shopping_germ
01286fa0   _n_ShotTone1
01285fbc   _n_ShotTone1_e
01286888   _n_ShotTone1_fren
012863f0   _n_ShotTone1_germ
01286fc0   _n_ShotTone2
01285fd4   _n_ShotTone2_e
012868a0   _n_ShotTone2_fren
01286408   _n_ShotTone2_germ
01286fe0   _n_ShotTone3
01285fec   _n_ShotTone3_e
012868b8   _n_ShotTone3_fren
01286420   _n_ShotTone3_germ
01287000   _n_ShotTone4
01286004   _n_ShotTone4_e
012868d0   _n_ShotTone4_fren
01286438   _n_ShotTone4_germ
01287020   _n_ShotTone5
0128601c   _n_ShotTone5_e
012868e8   _n_ShotTone5_fren
01286450   _n_ShotTone5_germ
01286ec0   _n_Silent
01285f28   _n_Silent_e
01286860   _n_Silent_fren
012863cc   _n_Silent_germ
01286960   _n_Soul
01285bdc   _n_Soul_e
012864c8   _n_Soul_fren
0128607c   _n_Soul_germ
01286a20   _n_Speed
01285c40   _n_Speed_e
01286530   _n_Speed_fren
012860d8   _n_Speed_germ
01286a60   _n_SunnySamba
01285c64   _n_SunnySamba_e
01286554   _n_SunnySamba_fren
012860fc   _n_SunnySamba_germ
01286b40   _n_Swan
01285d1c   _n_Swan_e
0128660c   _n_Swan_fren
012861b4   _n_Swan_germ
01286be0   _n_TheDollsDream
01285d90   _n_TheDollsDream_e
01286680   _n_TheDollsDream_fren
01286228   _n_TheDollsDream_germ
01286b80   _n_TwelveDays
01285d3c   _n_TwelveDays_e
0128662c   _n_TwelveDays_fren
012861d4   _n_TwelveDays_germ
01286ee0   _n_Vibrator_1
01285f38   _n_Vibrator_1_e
01286864   _n_Vibrator_1_fren
012863d0   _n_Vibrator_1_germ
01286f00   _n_Vibrator_2
01285f50   _n_Vibrator_2_e
01286868   _n_Vibrator_2_fren
012863d4   _n_Vibrator_2_germ
01286f20   _n_Vibrator_3
01285f68   _n_Vibrator_3_e
0128686c   _n_Vibrator_3_fren
012863d8   _n_Vibrator_3_germ
01286f40   _n_Vibrator_4
01285f80   _n_Vibrator_4_e
01286870   _n_Vibrator_4_fren
012863dc   _n_Vibrator_4_germ
01286f60   _n_Vibrator_5
01285f98   _n_Vibrator_5_e
01286874   _n_Vibrator_5_fren
012863e0   _n_Vibrator_5_germ
01286900   _n_aroundtheworld
01285b90   _n_aroundtheworld_e
01286468   _n_aroundtheworld_fren
01286034   _n_aroundtheworld_germ
01286980   _n_straightway
01285be8   _n_straightway_e
012864d4   _n_straightway_fren
01286088   _n_straightway_germ
0118760c   _norespTIL
01187afc   _numerrTIL
01195ef4   _objectTIL
01195c5c   _objinfoTIL
01198b20   _omaddTIL
01198edc   _omadoneTIL
01198d64   _omadwnldTIL
01198fc8   _omaerrorTIL
0119906c   _omawfaTIL
01197054   _omlaunchTIL
011963fc   _omsessTIL
01196e84   _omutcnfTIL
01196b74   _omutinpTIL
011965a4   _omutselTIL
01197130   _omutsselTIL
011969ec   _omutstatTIL
01199be0   _otabeginTIL
011999dc   _otadoneTIL
01199728   _otadwnldTIL
0119912c   _otajadTIL
01199a70   _otamsgTIL
01195188   _prmptdlgTIL
0119a094   _resCOMMON
01277ac8   _resDADK
0125a3bc   _resDEDE
012827b0   _resEN
0126c474   _resFIFI
012606e0   _resFRFR
012666bc   _resNLNL
0127d374   _resNONO
012720e4   _resSVSE
01194ba4   _returnTIL
0118c100   _rootcertTIL
011921e4   _saveasTIL
011926bc   _saveconfTIL
01192618   _saveerrTIL
01192598   _saveinfoTIL
01188c08   _scrlmodeTIL
011885a4   _scrtmenuTIL
01188904   _scrtprmpTIL
01189414   _setrepstTIL
0118b304   _shortcutTIL
01188830   _showcertTIL
01195514   _showurlTIL
0118c56c   _slmodeTIL
01194200   _snapccfmTIL
01194ac4   _snapconfTIL
01193ff4   _snapdispTIL
01194754   _snapdlstTIL
01194330   _snapdtlsTIL
01193d9c   _snapgoTIL
01192ff8   _snaplistTIL
01192e84   _snapmenuTIL
01194600   _snapourlTIL
011939d0   _snapresuTIL
011937c0   _snaptitlTIL
01195950   _softmenuTIL
01192cfc   _soundTIL
011895e8   _splashTIL
0118bd40   _srchinptTIL
01187c38   _svrpickTIL
01196148   _symtabTIL
01187c00   _syserrTIL
011875a8   _syspopupTIL
01192994   _timeoutTIL
01192b68   _title_rTIL
0118ba18   _toolmenuTIL
01287f04   _wap_UserLabel_Danish
01287a6c   _wap_UserLabel_Dutch
01287b90   _wap_UserLabel_English
01287cc0   _wap_UserLabel_Finnish
012877f8   _wap_UserLabel_French
01287938   _wap_UserLabel_German
01288020   _wap_UserLabel_Norwegian
01287de4   _wap_UserLabel_Swedish
01195478   _wapprovTIL
01195ed8   _wrapTIL
011957fc   _wwwinputTIL
0128817c   etext


GLOBAL SYMBOLS: SORTED BY Symbol Address 

address    name
--------   ----
01170000   _LanguagePack
01170028   _lp_Finnish_Dict
01187578   _blankTIL
011875a8   _syspopupTIL
0118760c   _norespTIL
01187afc   _numerrTIL
01187b8c   _apperrTIL
01187c00   _syserrTIL
01187c38   _svrpickTIL
01187e0c   _homepickTIL
01187ebc   _entrhomeTIL
01188358   _altsettTIL
011885a4   _scrtmenuTIL
01188830   _showcertTIL
01188904   _scrtprmpTIL
01188b0c   _cookiclrTIL
01188c08   _scrlmodeTIL
01188ec0   _cryptTIL
0118918c   _keycheckTIL
01189200   _keytimeTIL
01189414   _setrepstTIL
011895e8   _splashTIL
0118967c   _advancedTIL
0118980c   _aboutTIL
01189a68   _aboutsslTIL
01189ed0   _alertTIL
0118a0d0   _alert_0TIL
0118a30c   _alert_imTIL
0118a4ec   _aspawnTIL
0118a584   _authTIL
0118a778   _histnavTIL
0118ab38   _histlistTIL
0118af58   _bawalletTIL
0118b110   _homeexitTIL
0118b20c   _homesvdTIL
0118b304   _shortcutTIL
0118b50c   _advdmenuTIL
0118b6f0   _altadvdTIL
0118ba18   _toolmenuTIL
0118bb6c   _clearTIL
0118bd40   _srchinptTIL
0118be2c   _clearpopTIL
0118bfb0   _histpopTIL
0118c100   _rootcertTIL
0118c230   _intrlcssTIL
0118c280   _dialogTIL
0118c4dc   _drmmsgTIL
0118c56c   _slmodeTIL
0118c73c   _bkmkmenuTIL
0118c7e0   _booknewTIL
0118cadc   _booksavdTIL
0118cc28   _bookwrapTIL
0118ccb8   _booktopTIL
0118d590   _bookdelTIL
0118d708   _bookerrTIL
0118d82c   _bookgoTIL
0118da5c   _booknewfTIL
0118dd24   _bookfolTIL
0118e398   _bookccfmTIL
0118e4b8   _bookmoveTIL
0118e784   _bookdelaTIL
0118e978   _bookmkpgTIL
0118ec28   _bookstfTIL
0118ef20   _booktphkTIL
0118f308   _bookflhkTIL
0118f620   _bookhtkyTIL
0118fa18   _bookstnfTIL
0118fbcc   _bookmtnfTIL
0118fd74   _bookdtlTIL
0118ff18   _booktpdlTIL
01190318   _bookfldlTIL
01190604   _bookfullTIL
01190764   _bookmmsgTIL
01190888   _bookffulTIL
011909c4   _bookfdlsTIL
01190c1c   _bookccf2TIL
01190d98   _booknomkTIL
01190f18   _bookmvflTIL
01191320   _bookmvtpTIL
0119185c   _bookpassTIL
01191988   _bookpserTIL
01191ad4   _booksaveTIL
01191d24   _bktbmptyTIL
01191e8c   _bookpostTIL
01191fd8   _bookinpoTIL
01192124   _markcss2TIL
011921e4   _saveasTIL
01192598   _saveinfoTIL
01192618   _saveerrTIL
011926bc   _saveconfTIL
0119279c   _httprefTIL
01192994   _timeoutTIL
01192b68   _title_rTIL
01192cfc   _soundTIL
01192e84   _snapmenuTIL
01192ff8   _snaplistTIL
011937c0   _snaptitlTIL
011939d0   _snapresuTIL
01193d9c   _snapgoTIL
01193ff4   _snapdispTIL
01194200   _snapccfmTIL
01194330   _snapdtlsTIL
01194600   _snapourlTIL
01194754   _snapdlstTIL
01194ac4   _snapconfTIL
01194ba4   _returnTIL
01194c24   _cctprmptTIL
01194e28   _cctlingrTIL
011950b4   _loopTIL
01195114   _alertdlgTIL
01195188   _prmptdlgTIL
0119522c   _confdlgTIL
011952f0   _mmcconfmTIL
01195390   _mmcdispTIL
011953dc   _mmccomptTIL
01195428   _mmcerrorTIL
01195478   _wapprovTIL
01195514   _showurlTIL
011955d0   _gotourlTIL
011957fc   _wwwinputTIL
01195950   _softmenuTIL
01195978   _imgmenuTIL
01195ac4   _imginfoTIL
01195c5c   _objinfoTIL
01195dc8   _imageTIL
01195e24   _imgdispTIL
01195ed8   _wrapTIL
01195ef4   _objectTIL
01196070   _httperrTIL
011960a8   _e2einvalTIL
011960e0   _e2eexpTIL
01196148   _symtabTIL
01196180   _dldoneTIL
01196218   _dlerrorTIL
01196284   _dlpromptTIL
01196350   _dlprogresTIL
011963b8   _dlerror2TIL
011963fc   _omsessTIL
011965a4   _omutselTIL
011969ec   _omutstatTIL
01196b74   _omutinpTIL
01196e84   _omutcnfTIL
01197054   _omlaunchTIL
01197130   _omutsselTIL
011975e0   _mmsImmRetrievalTIL
011976a8   _mmssplashTIL
01197774   _certinfoTIL
011979f4   _certnoneTIL
01197b78   _certerbTIL
01197e74   _certerb0TIL
01197fbc   _camgmtTIL
0119867c   _connprmtTIL
0119887c   _connsec0TIL
0119895c   _connsec1TIL
01198a30   _connsec2TIL
01198b20   _omaddTIL
01198d64   _omadwnldTIL
01198edc   _omadoneTIL
01198fc8   _omaerrorTIL
0119906c   _omawfaTIL
0119912c   _otajadTIL
01199728   _otadwnldTIL
011999dc   _otadoneTIL
01199a70   _otamsgTIL
01199be0   _otabeginTIL
01199f14   _devpopupTIL
01199f84   _devpopu1TIL
01199fcc   _devpulldTIL
0119a094   _resCOMMON
0119a5d4   _lp_Swedish_Dict
011a832c   _lp_Norwegian_Dict
011b601c   _lp_Danish_Dict
011c3cf8   _lp_Dutch_Dict
011d19a4   _lp_German_Dict
011ddd34   _lp_Latin_Font
011f56d0   _lp_Finnish_Text
01200c28   _lp_German_Text
01200c34   _lp_French_Dict
01217294   _lp_French_Text
012222c4   _lp_Dutch_Text
0122cc84   _lp_Swedish_Text
01237600   _lp_Norwegian_Text
01241e9c   _lp_Danish_Text
0124c0c0   _lp_English_Text
0124c0cc   _lp_English_Dict
0125a3bc   _resDEDE
012606e0   _resFRFR
012666bc   _resNLNL
0126c474   _resFIFI
012720e4   _resSVSE
01277ac8   _resDADK
0127d374   _resNONO
012827b0   _resEN
01283c48   _n_EMS_Flirty_e
01283c70   _n_EMS_Glad_e
01283c84   _n_EMS_Sceptic_e
01283ca0   _n_EMS_Sad_e
01283cb4   _n_EMS_Wow_e
01283cc0   _n_EMS_Crying_e
01283cd8   _n_EMS_Winking_e
01283cf4   _n_EMS_Laughing_e
01283d10   _n_EMS_Indifferent_e
01283d34   _n_EMS_Kissing_e
01283d54   _n_EMS_Confused_e
01283d70   _n_EMS_Tongue_e
01283d98   _n_EMS_Angry_e
01283db0   _n_EMS_Glasses_e
01283dd0   _n_EMS_Devil_e
01283ddc   _n_EMS_NoDefPic_e
01283df4   _n_EMS_NoDefAnim_e
01283e10   _n_EMS_NoDefSound_e
01283e24   _n_EMS_Star_e
01283e30   _n_EMS_Paw_e
01283e38   _n_EMS_TurnAround_e
01283e50   _n_COM_Wallpaper1_e
01283e64   _n_COM_Wallpaper2_e
01283e7c   _n_COM_Wallpaper3_e
01283e90   _n_COM_Wallpaper4_e
01283ea4   _n_COM_Wallpaper5_e
01283eb0   _n_SHRCT_Boy_e
01283eb8   _n_SHRCT_Brother_e
01283ec8   _n_SHRCT_Father_e
01283ed8   _n_SHRCT_Girl_e
01283ee4   _n_SHRCT_Grandma_e
01283ef4   _n_SHRCT_Grandpa_e
01283f04   _n_SHRCT_Man_e
01283f0c   _n_SHRCT_Mother_e
01283f1c   _n_SHRCT_Nobody_e
01283f2c   _n_SHRCT_Sister_e
01283f3c   _n_SHRCT_Woman_e
01283f48   _n_EMS_Flirty_germ
01283f78   _n_EMS_Glad_germ
01283f98   _n_EMS_Sceptic_germ
01283fbc   _n_EMS_Sad_germ
01283fdc   _n_EMS_Wow_germ
01283fe8   _n_EMS_Crying_germ
01283ffc   _n_EMS_Winking_germ
01284018   _n_EMS_Laughing_germ
0128402c   _n_EMS_Indifferent_germ
01284048   _n_EMS_Kissing_germ
01284068   _n_EMS_Confused_germ
0128408c   _n_EMS_Tongue_germ
012840b4   _n_EMS_Angry_germ
012840d4   _n_EMS_Glasses_germ
012840f0   _n_EMS_Devil_germ
01284100   _n_EMS_NoDefPic_germ
01284118   _n_EMS_NoDefAnim_germ
01284134   _n_EMS_NoDefSound_germ
01284148   _n_EMS_Star_germ
01284154   _n_EMS_Paw_germ
01284160   _n_EMS_TurnAround_germ
01284174   _n_COM_Wallpaper1_germ
01284188   _n_COM_Wallpaper2_germ
012841a0   _n_COM_Wallpaper3_germ
012841b4   _n_COM_Wallpaper4_germ
012841c8   _n_COM_Wallpaper5_germ
012841d4   _n_SHRCT_Boy_germ
012841dc   _n_SHRCT_Brother_germ
012841ec   _n_SHRCT_Father_germ
012841fc   _n_SHRCT_Girl_germ
01284208   _n_SHRCT_Grandma_germ
01284218   _n_SHRCT_Grandpa_germ
01284228   _n_SHRCT_Man_germ
01284230   _n_SHRCT_Mother_germ
01284240   _n_SHRCT_Nobody_germ
01284250   _n_SHRCT_Sister_germ
01284260   _n_SHRCT_Woman_germ
0128426c   _n_EMS_Flirty_fren
01284280   _n_EMS_Glad_fren
01284290   _n_EMS_Sceptic_fren
012842a4   _n_EMS_Sad_fren
012842b4   _n_EMS_Wow_fren
012842c4   _n_EMS_Crying_fren
012842d4   _n_EMS_Winking_fren
012842f8   _n_EMS_Laughing_fren
01284304   _n_EMS_Indifferent_fren
0128431c   _n_EMS_Kissing_fren
01284344   _n_EMS_Confused_fren
01284358   _n_EMS_Tongue_fren
01284374   _n_EMS_Angry_fren
01284380   _n_EMS_Glasses_fren
01284394   _n_EMS_Devil_fren
012843a4   _n_EMS_NoDefPic_fren
012843bc   _n_EMS_NoDefAnim_fren
012843d8   _n_EMS_NoDefSound_fren
012843ec   _n_EMS_Star_fren
012843fc   _n_EMS_Paw_fren
01284408   _n_EMS_TurnAround_fren
01284428   _n_COM_Wallpaper1_fren
0128443c   _n_COM_Wallpaper2_fren
01284454   _n_COM_Wallpaper3_fren
01284468   _n_COM_Wallpaper4_fren
0128447c   _n_COM_Wallpaper5_fren
01284488   _n_SHRCT_Boy_fren
01284490   _n_SHRCT_Brother_fren
012844a0   _n_SHRCT_Father_fren
012844b0   _n_SHRCT_Girl_fren
012844bc   _n_SHRCT_Grandma_fren
012844cc   _n_SHRCT_Grandpa_fren
012844dc   _n_SHRCT_Man_fren
012844e4   _n_SHRCT_Mother_fren
012844f4   _n_SHRCT_Nobody_fren
01284504   _n_SHRCT_Sister_fren
01284514   _n_SHRCT_Woman_fren
01284520   _n_EMS_Flirty
01284540   _n_EMS_Glad
01284560   _n_EMS_Sceptic
01284580   _n_EMS_Sad
012845a0   _n_EMS_Wow
012845c0   _n_EMS_Crying
012845e0   _n_EMS_Winking
01284600   _n_EMS_Laughing
01284620   _n_EMS_Indifferent
01284640   _n_EMS_Kissing
01284660   _n_EMS_Confused
01284680   _n_EMS_Tongue
012846a0   _n_EMS_Angry
012846c0   _n_EMS_Glasses
012846e0   _n_EMS_Devil
01284700   _n_EMS_NoDefPic
01284720   _n_EMS_NoDefAnim
01284740   _n_EMS_NoDefSound
01284760   _n_EMS_Star
01284780   _n_EMS_Paw
012847a0   _n_EMS_TurnAround
012847c0   _n_COM_Wallpaper1
012847e0   _n_COM_Wallpaper2
01284800   _n_COM_Wallpaper3
01284820   _n_COM_Wallpaper4
01284840   _n_COM_Wallpaper5
01284860   _n_SHRCT_Boy
01284880   _n_SHRCT_Brother
012848a0   _n_SHRCT_Father
012848c0   _n_SHRCT_Girl
012848e0   _n_SHRCT_Grandma
01284900   _n_SHRCT_Grandpa
01284920   _n_SHRCT_Man
01284940   _n_SHRCT_Mother
01284960   _n_SHRCT_Nobody
01284980   _n_SHRCT_Sister
012849a0   _n_SHRCT_Woman
012849c0   _ml_imageNameLib
01285b90   _n_aroundtheworld_e
01285bb4   _n_BenQisComing_e
01285bc8   _n_DownHome_e
01285bdc   _n_Soul_e
01285be8   _n_straightway_e
01285c04   _n_Fly_e
01285c0c   _n_Shopping_e
01285c20   _n_Fire_e
01285c2c   _n_LadyMary_e
01285c40   _n_Speed_e
01285c4c   _n_Friendship_e
01285c64   _n_SunnySamba_e
01285c7c   _n_Breeze_e
01285c8c   _n_Dance_e
01285c98   _n_Papillon_e
01285cac   _n_GlistensTheQuartz_e
01285cd4   _n_GrandfathersClock_e
01285cfc   _n_RedIsTheRose_e
01285d1c   _n_Swan_e
01285d28   _n_Nostalgia_e
01285d3c   _n_TwelveDays_e
01285d54   _n_BeautifulGirls_e
01285d74   _n_GreatPalace_e
01285d90   _n_TheDollsDream_e
01285db4   _n_Alert_1_e
01285dc4   _n_Alert_2_e
01285dd4   _n_Alert_3_e
01285de4   _n_Alert_4_e
01285df4   _n_Alert_5_e
01285e04   _n_Alert_6_e
01285e14   _n_Alert_7_e
01285e24   _n_Alert_8_e
01285e34   _n_Alert_9_e
01285e44   _n_Alert_10_e
01285e58   _n_Alert_11_e
01285e6c   _n_Alert_12_e
01285e80   _n_EMS_Chimes_High_e
01285e98   _n_EMS_Chimes_Low_e
01285eb0   _n_EMS_Ding_e
01285ebc   _n_EMS_Tada_e
01285ec8   _n_EMS_Notify_e
01285ed8   _n_EMS_Drum_e
01285ee4   _n_EMS_Claps_e
01285ef0   _n_EMS_Fanfare_e
01285f00   _n_EMS_ChordHigh_e
01285f14   _n_EMS_ChordLow_e
01285f28   _n_Silent_e
01285f38   _n_Vibrator_1_e
01285f50   _n_Vibrator_2_e
01285f68   _n_Vibrator_3_e
01285f80   _n_Vibrator_4_e
01285f98   _n_Vibrator_5_e
01285fb0   _n_EMS_Bugle_e
01285fbc   _n_ShotTone1_e
01285fd4   _n_ShotTone2_e
01285fec   _n_ShotTone3_e
01286004   _n_ShotTone4_e
0128601c   _n_ShotTone5_e
01286034   _n_aroundtheworld_germ
01286058   _n_BenQisComing_germ
01286068   _n_DownHome_germ
0128607c   _n_Soul_germ
01286088   _n_straightway_germ
0128609c   _n_Fly_germ
012860a4   _n_Shopping_germ
012860b8   _n_Fire_germ
012860c4   _n_LadyMary_germ
012860d8   _n_Speed_germ
012860e4   _n_Friendship_germ
012860fc   _n_SunnySamba_germ
01286114   _n_Breeze_germ
01286124   _n_Dance_germ
01286130   _n_Papillon_germ
01286144   _n_GlistensTheQuartz_germ
0128616c   _n_GrandfathersClock_germ
01286194   _n_RedIsTheRose_germ
012861b4   _n_Swan_germ
012861c0   _n_Nostalgia_germ
012861d4   _n_TwelveDays_germ
012861ec   _n_BeautifulGirls_germ
0128620c   _n_GreatPalace_germ
01286228   _n_TheDollsDream_germ
0128624c   _n_Alert_1_germ
0128625c   _n_Alert_2_germ
0128626c   _n_Alert_3_germ
0128627c   _n_Alert_4_germ
0128628c   _n_Alert_5_germ
0128629c   _n_Alert_6_germ
012862ac   _n_Alert_7_germ
012862bc   _n_Alert_8_germ
012862cc   _n_Alert_9_germ
012862dc   _n_Alert_10_germ
012862f0   _n_Alert_11_germ
01286304   _n_Alert_12_germ
01286318   _n_EMS_Chimes_High_germ
01286330   _n_EMS_Chimes_Low_germ
01286348   _n_EMS_Ding_germ
01286354   _n_EMS_Tada_germ
01286360   _n_EMS_Notify_germ
01286370   _n_EMS_Drum_germ
01286380   _n_EMS_Claps_germ
01286394   _n_EMS_Fanfare_germ
012863a4   _n_EMS_ChordHigh_germ
012863b8   _n_EMS_ChordLow_germ
012863cc   _n_Silent_germ
012863d0   _n_Vibrator_1_germ
012863d4   _n_Vibrator_2_germ
012863d8   _n_Vibrator_3_germ
012863dc   _n_Vibrator_4_germ
012863e0   _n_Vibrator_5_germ
012863e4   _n_EMS_Bugle_germ
012863f0   _n_ShotTone1_germ
01286408   _n_ShotTone2_germ
01286420   _n_ShotTone3_germ
01286438   _n_ShotTone4_germ
01286450   _n_ShotTone5_germ
01286468   _n_aroundtheworld_fren
01286488   _n_BenQisComing_fren
0128649c   _n_DownHome_fren
012864c8   _n_Soul_fren
012864d4   _n_straightway_fren
012864f4   _n_Fly_fren
012864fc   _n_Shopping_fren
01286510   _n_Fire_fren
0128651c   _n_LadyMary_fren
01286530   _n_Speed_fren
0128653c   _n_Friendship_fren
01286554   _n_SunnySamba_fren
0128656c   _n_Breeze_fren
0128657c   _n_Dance_fren
01286588   _n_Papillon_fren
0128659c   _n_GlistensTheQuartz_fren
012865c4   _n_GrandfathersClock_fren
012865ec   _n_RedIsTheRose_fren
0128660c   _n_Swan_fren
01286618   _n_Nostalgia_fren
0128662c   _n_TwelveDays_fren
01286644   _n_BeautifulGirls_fren
01286664   _n_GreatPalace_fren
01286680   _n_TheDollsDream_fren
012866a4   _n_Alert_1_fren
012866b8   _n_Alert_2_fren
012866cc   _n_Alert_3_fren
012866e0   _n_Alert_4_fren
012866f4   _n_Alert_5_fren
01286708   _n_Alert_6_fren
0128671c   _n_Alert_7_fren
01286730   _n_Alert_8_fren
01286744   _n_Alert_9_fren
01286758   _n_Alert_10_fren
0128676c   _n_Alert_11_fren
01286780   _n_Alert_12_fren
01286794   _n_EMS_Chimes_High_fren
012867b4   _n_EMS_Chimes_Low_fren
012867d0   _n_EMS_Ding_fren
012867dc   _n_EMS_Tada_fren
012867e8   _n_EMS_Notify_fren
012867fc   _n_EMS_Drum_fren
01286810   _n_EMS_Claps_fren
01286824   _n_EMS_Fanfare_fren
01286834   _n_EMS_ChordHigh_fren
0128684c   _n_EMS_ChordLow_fren
01286860   _n_Silent_fren
01286864   _n_Vibrator_1_fren
01286868   _n_Vibrator_2_fren
0128686c   _n_Vibrator_3_fren
01286870   _n_Vibrator_4_fren
01286874   _n_Vibrator_5_fren
01286878   _n_EMS_Bugle_fren
01286888   _n_ShotTone1_fren
012868a0   _n_ShotTone2_fren
012868b8   _n_ShotTone3_fren
012868d0   _n_ShotTone4_fren
012868e8   _n_ShotTone5_fren
01286900   _n_aroundtheworld
01286920   _n_BenQisComing
01286940   _n_DownHome
01286960   _n_Soul
01286980   _n_straightway
012869a0   _n_Fly
012869c0   _n_Shopping
012869e0   _n_Fire
01286a00   _n_LadyMary
01286a20   _n_Speed
01286a40   _n_Friendship
01286a60   _n_SunnySamba
01286a80   _n_Breeze
01286aa0   _n_Dance
01286ac0   _n_Papillon
01286ae0   _n_GlistensTheQuartz
01286b00   _n_GrandfathersClock
01286b20   _n_RedIsTheRose
01286b40   _n_Swan
01286b60   _n_Nostalgia
01286b80   _n_TwelveDays
01286ba0   _n_BeautifulGirls
01286bc0   _n_GreatPalace
01286be0   _n_TheDollsDream
01286c00   _n_Alert_1
01286c20   _n_Alert_2
01286c40   _n_Alert_3
01286c60   _n_Alert_4
01286c80   _n_Alert_5
01286ca0   _n_Alert_6
01286cc0   _n_Alert_7
01286ce0   _n_Alert_8
01286d00   _n_Alert_9
01286d20   _n_Alert_10
01286d40   _n_Alert_11
01286d60   _n_Alert_12
01286d80   _n_EMS_Chimes_High
01286da0   _n_EMS_Chimes_Low
01286dc0   _n_EMS_Ding
01286de0   _n_EMS_Tada
01286e00   _n_EMS_Notify
01286e20   _n_EMS_Drum
01286e40   _n_EMS_Claps
01286e60   _n_EMS_Fanfare
01286e80   _n_EMS_ChordHigh
01286ea0   _n_EMS_ChordLow
01286ec0   _n_Silent
01286ee0   _n_Vibrator_1
01286f00   _n_Vibrator_2
01286f20   _n_Vibrator_3
01286f40   _n_Vibrator_4
01286f60   _n_Vibrator_5
01286f80   _n_EMS_Bugle
01286fa0   _n_ShotTone1
01286fc0   _n_ShotTone2
01286fe0   _n_ShotTone3
01287000   _n_ShotTone4
01287020   _n_ShotTone5
01287040   _ml_melodyNameLib
01287144   _IME_MODULES
012874b4   _lp_Global_ResList
012874e4   _lp_Global_LangResList
012874f0   _lp_English_ResList
01287520   _LANG_INFO_ENGLISH
01287530   _lp_German_ResList
01287560   _LANG_INFO_GERMAN
01287570   _lp_French_ResList
012875a0   _LANG_INFO_FRENCH
012875b0   _lp_Dutch_ResList
012875e0   _LANG_INFO_DUTCH
012875f0   _lp_Swedish_ResList
01287620   _LANG_INFO_SWEDISH
01287630   _lp_Danish_ResList
01287660   _LANG_INFO_DANISH
01287670   _lp_Finnish_ResList
012876a0   _LANG_INFO_FINNISH
012876b0   _lp_Norwegian_ResList
012876e0   _LANG_INFO_NORWEGIAN
012877f8   _wap_UserLabel_French
01287938   _wap_UserLabel_German
01287a6c   _wap_UserLabel_Dutch
01287b90   _wap_UserLabel_English
01287cc0   _wap_UserLabel_Finnish
01287de4   _wap_UserLabel_Swedish
01287f04   _wap_UserLabel_Danish
01288020   _wap_UserLabel_Norwegian
01288068   _lp_CP1252_Encode
012880fc   _lp_CP1252_Decode
0128817c   .text
0128817c   ___etext__
0128817c   ___text__
0128817c   etext
01330000   _i_EMS_Flirty
01330c0c   _i_EMS_Glad
01331818   _i_EMS_Sceptic
01332424   _i_EMS_Sad
01333030   _i_EMS_Wow
01333c3c   _i_EMS_Crying
01334848   _i_EMS_Winking
01335454   _i_EMS_Laughing
01336060   _i_EMS_Indifferent
01336c6c   _i_EMS_Kissing
01337878   _i_EMS_Confused
01338484   _i_EMS_Tongue
01339090   _i_EMS_Angry
01339c9c   _i_EMS_Glasses
0133a8a8   _i_EMS_Devil
0133b4b4   _i_EMS_NoDefPic
0133b7c0   _i_EMS_NoDefAnim
0133bacc   _i_EMS_NoDefSound
0133bb98   _i_EMS_Star
0133bea4   _i_EMS_Paw
0133c1b0   _i_EMS_TurnAround
015417f4   _ml_imageLib
015429c4   _i_aroundtheworld
01545728   _i_BenQisComing
01546694   _i_DownHome
01548814   _i_Soul
0154b6e0   _i_straightway
0154ce48   _i_Fly
0154fbc0   _i_Shopping
0155433c   _i_Fire
01555934   _i_LadyMary
01557824   _i_Speed
01559e7c   _i_Friendship
0155fb9c   _i_SunnySamba
01562ca8   _i_Breeze
0156478c   _i_Dance
015680dc   _i_Papillon
01569788   _i_Alert_1
0156984c   _i_Alert_2
01569958   _i_Alert_3
01569b38   _i_Alert_4
01569f64   _i_Alert_5
0156a070   _i_Alert_6
0156a314   _i_Alert_7
0156a3d8   _i_Alert_8
0156a7e8   _i_Alert_9
0156a900   _i_Alert_10
0156ab08   _i_Alert_11
0156ac5c   _i_Alert_12
0156ad74   _i_ShotTone_Multishot
0156b3bc   _i_Camera_Record_End
0156c574   _i_Camera_Record_Start
0156d72c   _i_SelfTimer_1Seconds1beat
0156e58c   _i_SelfTimer_1Seconds3beat
015704d8   _i_Power_Up
01570754   _i_Power_Down
0157084c   _i_CMR_Timer_Short
01570924   _i_CMR_Timer_Long
01570a74   _i_CMR_MutiShot
01570ebc   _i_Vedio_Record_Start
01570f38   _i_Vedio_Record_End
01570fc4   _i_Accessary_In
01571094   _i_Battery_Low
015711a8   _i_Call_Start
01571220   _i_Network_On
01571308   _i_EMS_Chimes_High
015713a0   _i_EMS_Chimes_Low
0157143c   _i_EMS_Ding
015714bc   _i_EMS_Tada
01571538   _i_EMS_Notify
015715c4   _i_EMS_Drum
0157165c   _i_EMS_Claps
015716e8   _i_EMS_Fanfare
01571770   _i_EMS_ChordHigh
015717f4   _i_EMS_ChordLow
01571874   _i_EMS_Bugle
015718f8   _i_ShotTone1
01571900   _i_ShotTone2
01571908   _i_ShotTone3
01571910   _i_ShotTone4
01571918   _i_ShotTone5
01571920   _ml_melodyLib
UNDEFED _c_int00

[691 symbols]
